:10411500000A0014000500320032000A0005000AFA
:02412500C35085
:103B7300C10B4101970101C901013800012800016E
:103B83003D00013F00012500012B00012D00C10A6A
:103B9300C1000123FF41013F0041017400014300C3
:0E3BA300C103C182C108012A00014200C10114
:1032FA00E4F544F545F5A0F590F5D81218009001CB
:10330A003F7403F0124041123ED5AF23123FC23040
:10331A000926C2097874E6600B16E6B40106200590
:10332A00031217CEE568D39400400DD5680A1241FE
:10333A00667F0A7E0012414F78A9E6D39403405073
:10334A00E4F612418512393FE4F541E54125E024CE
:10335A00B7F8E6FE08E6FF900198EEF0A3EFF04E0C
:10336A006025E024FFF0900198E034FFF0E0FEA32E
:10337A00E0FFE54125E024B7F8A60608A607EF4EC8
:10338A007005AF411241030541E541C3940940BBB1
:10339A00E538700261191538742F2538F8E614607B
:1033AA002B146032147002813924FC70028140149B
:1033BA0070028154240870D80545E545C3940A4033
:1033CA0005E4F545B204E4FDFCFF8079120800E447
:1033DA00FDFC7F01806FE51C7003123ED53013217E
:1033EA00C213E4F54490011DE0FF123F9B40397F70
:1033FA00057E0012414F0544E544C3940540E6802A
:10340A0027301221C212E4F54490011BE0FF123F5B
:10341A00C240157F057E0012414F0544E544C3941E
:10342A000540E6800312405FE4FDFC7F028016E45B
:10343A00FDFC7F03800FA20BE433FF121C5BB20B6F
:10344A00E4FDFC7F07123EA0619A122A2A123E9BD3
:02345A00619A75
:10180000E4F580124127900050741EF0E49001AA84
:10181000F09001AAE0FFC39408501DEF25E025E0F9
:101820002462F582E43400F58312152500000000DF
:101830009001AAE004F080D97B017A0179ACE4F54B
:10184000537F15121F08500221017B017A0179ACE8
:10185000E4F5537F16121F084052E49001ACF0A348
:10186000F09001AAF09001AAE0FFC3941040022179
:1018700054EF2415FF9001ACE0FCA3E0FDE4FB1263
:101880003CD59001AAE025E0FFE433FE74D22FF5A9
:101890008274003EF583E4F074D32FF58274003E29
:1018A000F583E4F09001AAE004F080B9E49001AA85
:1018B000F09001AAE0FFC3941040022154EF2415D8
:1018C000FF7B017A0179ACE4F553121F089001AC5B
:1018D000E0FD9001AAE025E0FFE433FE74D22FF58D
:1018E0008274003EF583EDF09001ADE0FD74D32FDE
:1018F000F58274003EF583EDF09001AAE004F080DB
:10190000B0E49001AAF09001AAE0FFC39410504403
:10191000EF2415FF7B017A0179ACE4F553121F081F
:101920009001ACE0FD9001AAE025E0FFE433FE74F5
:10193000D22FF58274003EF583EDF09001ADE0FD0D
:1019400074D32FF58274003EF583EDF09001AAE088
:1019500004F080B2E49001AAF09001AAE0FFC394E1
:10196000205014741E2FF582E43401F583E4F090C6
:1019700001AAE004F080E29001AA7410F09001AA9C
:10198000E0FFC394385033E49001ACF0A3F0EF24AF
:1019900015FF7B017A0179ACE4F553121F08900121
:1019A000ADE0FF9001AAE024E2F582E43400F58383
:1019B000EFF09001AAE004F080C37B017A0179ACDA
:1019C000E4F5537F4D121F0840057523FF800690F4
:1019D00001ADE0F523E49001AAF09001AAE0FFC375
:1019E00094205052EF244EFF7B017A0179ACE4F54C
:1019F00053121F0840119001AAE024B2F582E4348A
:101A000000F583E4F08027D39001ADE094059001C8
:101A1000ACE094004004E4F0A3F09001ADE0FF904E
:101A200001AAE024B2F582E43400F583EFF09001DE
:101A3000AAE004F080A430001CD2A0D2A1D2A2D28D
:101A4000A3D2A4D2A5D2A6D2A7D290D291D292D21A
:101A500093D2DB801AC2A0C2A1C2A2C2A3C2A4C2F6
:101A6000A5C2A6C2A7C290C291C292C293C2DBD243
:101A7000B4D2B2D294D295C2B7C2B5C2B6C2DAC29B
:101A8000D9C2B37B017A0179ABE4F5547F0F123AE6
:101A9000E540069001AB7401F09001ABE0B4010B9E
:101AA00075878090011C7403F08009E4F58790012C
:101AB0001C7406F07580FF759850758921758DFD31
:101AC000758BFD758A04758CF7D28ED28CD2A943A2
:101AD000BF02123D87D2AFD2AC75270112418512E9
:101AE000414B12418512414B12418512414B12412B
:101AF0008512414B12418512414B124185E4F52775
:101B00009001AAF09001AAE0FFC3941A5018EF25A3
:101B1000E02440F582E43401F583E4F0A3F0900181
:101B2000AAE004F080DEE49001AAF09001AAE0FFB0
:101B3000C3940D500B74AA2FF8E4F6E004F080EB88
:101B4000E49001AAF09001AAE0FFC39409500FEFBE
:101B500025E024B7F8E4F608F6E004F080E7E4FBBB
:101B6000FDFC7F63123CD5E490013EF07B017A01DD
:101B70007995F5547F0D123AE540069001957480F1
:101B8000F07B017A017997E4F5547F0C123AE54035
:101B90000AE4FB7D01FC7F0C123CD5900197E070BC
:101BA0000FFB7D01FC7F0C123CD59001977401F076
:101BB000E4FB7D0EFC7F05123CD5E4FB7D14FC7F2D
:101BC00007123CD57B017A01793FE4F5547F081276
:101BD0003AE5E4FDFCFF123EA0E4FDFC7F02123E6C
:101BE000A0E4FDFC7F01123EA0E4FDFC7F07123E55
:101BF000A0900197E06402703BFDFC7F04123EA0C0
:101C0000E49001AAF09001AAE0FFC394105018EFED
:101C100025E02475F582E43401F583E4F0A3F09027
:101C200001AAE004F080DE90013EE030E704D20635
:101C30008002C206123E9BE49001AAF09001AAE045
:101C4000FFC39420501474922FF582E43400F5837E
:0A1C5000E4F09001AAE004F080E245
:011C5A002267
:03000B00023D3380
:103D3300C0E0C0F0C083C082C0D075D000C000C056
:103D430001C002C003C004C005C006C007758A04D1
:103D5300758CF778A906D2097580FF78C906E6D372
:103D6300940440027601123C70D007D006D005D0EF
:103D730004D003D002D001D000D0D0D082D083D0E1
:043D8300F0D0E0326A
:10410300E538C39409500AAE380538742F2EF8A643
:02411300072281
:053E9B00E4FDFC7F08BE
:103EA0008C508D51E5514550701FEF25E02415F5DC
:103EB00082E43441F583E493FC740193FDEF25E043
:103EC00024B7F8A60408A60522EF25E024B7F8A633
:053ED0005008A651227C
:1040410090013FE0FF7006439B4075A303EFC394CB
:0E405100014002D20AEFC394034002D20022C3
:10405F00E51CB40107D20C7F0802070BE51CB40264
:0D406F0003022F0AE51CB403031235B6222C
:021C5B008F46B2
:101C5D00E4F54AD20FE54614604104600281F58532
:101C6D008049A2B7920CA2B5920DA2B6920EA2DA3D
:101C7D009210C2B7C2B5C2B6C2DA7580FFC2B47FC8
:101C8D000A7E0012414FC294858047D2947580FF21
:101C9D00C295858048D295D2B4803A858049A2B745
:101CAD00920CA2B5920DA2B6920EA2DA9210C2B704
:101CBD00C2B5C2B6C2DA7580FFC2B27F0A7E00120B
:101CCD00414FC294858047D2947580FFC29585801F
:101CDD0048D295D2B2854980A20C92B7A20D92B589
:101CED00A20E92B6A21092DA7D01E4FCE5475D707A
:101CFD0003D38001C3500AE5485D70028001C340E3
:101D0D0003ED424AED25E0FD0CBC08E0743F25468D
:101D1D00F8E6654A6023742D2546F806742D254690
:101D2D00F8E6C3940A4019743F2546F8A64A742D67
:101D3D002546F8E4F6D20F8007742D2546F8E4F613
:101D4D0074282546F8E66547602374252546F80670
:101D5D0074252546F8E6C3940A401974282546F8DB
:101D6D00A64774252546F8E4F6D20F80077425257D
:101D7D0046F8E4F6743D2546F8E665486023742B75
:101D8D002546F806742B2546F8E6C3940A401974C7
:101D9D003D2546F8A648742B2546F8E4F6D20F806B
:101DAD0007742B2546F8E4F67D01200F02C1AAC267
:101DBD000FE5467074FC743F2546F8E65D700280B1
:101DCD002274282546F8E65D700874AA2CF8760171
:101DDD008017743D2546F8E65D700874AA2CF876D8
:101DED0002800674AA2CF8E4F6ED25E0FD0CBC0883
:101DFD00C5E4900160F0A3F0FC900160E0FEA3E06B
:101E0D007802C333CE33CED8F9FF900160EEF0A344
:101E1D00EFF074AA2CF8E6FBEB4FFF900160EEF0AB
:101E2D00A3EFF00CBC08D280747C08743F2546F8F3
:101E3D00E65D7002802274282546F8E65D70087410
:101E4D00AA2CF876018017743D2546F8E65D7008DA
:101E5D0074AA2CF87602800674AA2CF8E4F6ED2507
:101E6D00E0FD0CBC10C5E4900162F0A3F07C08907D
:101E7D000162E0FEA3E07802C333CE33CED8F9FF82
:101E8D00900162EEF0A3EFF074AA2CF8E6FBEB4F95
:101E9D00FF900162EEF0A3EFF00CBC10D290019711
:101EAD00E0FF7048E5467023900160E0FAA3E0FB87
:101EBD004A6010EB64AA7003EA64AA6006BA55077B
:101ECD00BB5504D2038025C2038021900162E0FA44
:101EDD00A3E0FB4A6010EB64AA7003EA64AA6006F3
:101EED00BA5507BB5504D2038002C203EFB4030AEF
:0A1EFD007C0D78AA7402F608DCFCE4
:011F070022B7
:102A2A00E4F5467B007A007923AF461240C740029C
:102A3A0061CC7A00796BAF461240C74002615EAF43
:102A4A0046123FE9E54625E02415FFC007E546752D
:102A5A00F004A4FDACF0241EF58274013CF583E079
:102A6A00FE741F2DF58274013CF583E07C0024007E
:102A7A00FDEC3EFCD007123CD5E54625E02416FFC6
:102A8A00C007E54675F004A4FDACF02420F5827475
:102A9A00013CF583E0FE74212DF58274013CF58337
:102AAA00E07C002400FDEC3EFCD007E4FB123CD5A0
:102ABA00E54675F005A424F2F582E43400F583E0D6
:102ACA00FD7C00E54675F005A42425FFE4FB123CD5
:102ADA00D5E54675F005A424F3F582E43400F583C0
:102AEA00E0FD7C00E54675F005A42426FFE4FB1210
:102AFA003CD5E54675F005A424F4F582E43400F5E6
:102B0A0083E0FD7C00E54675F005A42427FFE4FB7D
:102B1A00123CD5E54675F005A424F5F582E43400A7
:102B2A00F583E0FD7C00E54675F005A42428FFE462
:102B3A00FB123CD5E54675F005A424F6F582E4348B
:102B4A0000F583E0FD7C00E54675F005A42429FF25
:102B5A00E4FB806BE54625E02415FFC007E54675D2
:102B6A00F004A4FDACF0241EF58274013CF583E068
:102B7A00FE741F2DF58274013CF583E07C0024006D
:102B8A00FDEC3EFCD007E4FB123CD5E54625E024EB
:102B9A0016FFC007E54675F004A4FDACF02420F545
:102BAA008274013CF583E0FE74212DF58274013CA8
:102BBA00F583E07C002400FDEC3EFCD007E4FB1228
:0D2BCA003CD50546E546C394085002412D58
:012BD70022DB
:10393F00900197E07012300405533AFE8003433A2A
:10394F000130031D80168019300405533AFE8003A1
:10395F00433A01E524D3940040071524533AFD80E0
:10396F0003433A02E539C31330A004F53980044408
:10397F0080F539E539C31330A104F539800444804B
:10398F00F539E539C31330A204F53980044480F5C5
:10399F0039E539C31330A304F53980044480F53970
:1039AF00E539C31330A404F53980044480F539E5B3
:1039BF0039C31330A504F53980044480F539E5394E
:1039CF00C31330A604F53980044480F539E539C3B3
:1039DF001330A704F53980044480F539309005532E
:1039EF003CFE8003433CE1309105533CFD80034393
:1039FF003CE2309205533CFB8003433CE43093059B
:103A0F00533CF78003433CE830DB05533CEF800326
:103A1F00433CF0E4FFEF25E02400F582E43400F5A9
:103A2F0083E0FCA3E0D39400EC9402E53B40051344
:0E3A3F00F53B8006C3134480F53B0FBF08D74C
:013A4D002256
:103C700078C9E624FE601F14603114604324037089
:103C800053C2B5C2B6C2DAE5276005E4F580800309
:103C9000853980D2B722C2B7C2B6C2DAE52760053D
:103CA000E4F5808003853A80D2B522C2B7C2B5C29E
:103CB000DAE5276005E4F5808003853B80D2B622F3
:103CC000C2B7C2B5C2B6E5276005E4F580800385BA
:053CD0003C80D2DA2265
:04418500759FA72259
:04414B007F507EC360
:0B414F00EF1FAC0670011E4C70F62242
:10265F0000C1814001C0804101C0804100C1814063
:10266F0001C0804100C1814000C1814001C0804153
:10267F0001C0804100C1814000C1814001C0804143
:10268F0000C1814001C0804101C0804100C1814033
:10269F0001C0804100C1814000C1814001C0804123
:1026AF0000C1814001C0804101C0804100C1814013
:1026BF0000C1814001C0804101C0804100C1814003
:1026CF0001C0804100C1814000C1814001C08041F3
:1026DF0001C0804100C1814000C1814001C08041E3
:1026EF0000C1814001C0804101C0804100C18140D3
:1026FF0000C1814001C0804101C0804100C18140C3
:10270F0001C0804100C1814000C1814001C08041B2
:10271F0000C1814001C0804101C0804100C18140A2
:10272F0001C0804100C1814000C1814001C0804192
:10273F0001C0804100C1814000C1814001C0804182
:10274F0000C1814001C0804101C0804100C1814072
:10275F0000C0C101C30302C2C60607C705C5C40432
:10276F00CC0C0DCD0FCFCE0E0ACACB0BC90908C8A2
:10277F00D81819D91BDBDA1A1EDEDF1FDD1D1CDC92
:10278F0014D4D515D71716D6D21213D311D1D01002
:10279F00F03031F133F3F23236F6F737F53534F4F2
:1027AF003CFCFD3DFF3F3EFEFA3A3BFB39F9F83862
:1027BF0028E8E929EB2B2AEAEE2E2FEF2DEDEC2C52
:1027CF00E42425E527E7E62622E2E323E12120E0C2
:1027DF00A06061A163A3A26266A6A767A56564A4B2
:1027EF006CACAD6DAF6F6EAEAA6A6BAB69A9A86822
:1027FF0078B8B979BB7B7ABABE7E7FBF7DBDBC7C12
:10280F00B47475B577B7B67672B2B373B17170B081
:10281F005090915193535292965657975595945471
:10282F009C5C5D9D5F9F9E5E5A9A9B5B99595898E1
:10283F00884849894B8B8A4A4E8E8F4F8D4D4C8CD1
:10284F004484854587474686824243834181804041
:103BB10041011C08017200C113C112016B000269AD
:063BC1000008026600127C
:1040B3007E01EEA807088002C333D8FCFE12121358
:0440C3004E0212593E
:103FE9007E01EEA807088002C333D8FCFE6306FFF2
:073FF9001212135E021259BF
:1040C7007E01EEA807088002C333D8FCFE12121344
:0340D7005E24FF65
:0140DA0022C3
:103D8700C2D8E47872F67874F6FB7A0079757F0604
:103D97007EEF12415A08E6FFF46003EF70167B00CE
:103DA7007A007975E4F5547F06123AE54013787581
:103DB70076FE80027875E6FD7C00E4FB7F06123C08
:0E3DC700D57875E66003B4FF04787576FE22A9
:0A416600C2D8E47872F67874F622ED
:05418000C211D2D8229B
:0300230002370C95
:10370C00C0E0C083C082C0D075D000C000C005C06E
:10371C00063098797872E6C394325007E60624771F
:10372C00F8A699C29890011CE0F5687872E6FD64E1
:10373C000770347878E6FE6403600DEEB406028000
:10374C0007EEB4100B20140890011A7408F0804492
:10375C00EEB4100B787DE6240990011AF0803590B8
:10376C00011A7432F0802D90011AE0B5050B7568C2
:10377C000078747606D214801B7872E6B403157840
:10378C0078E6B4190F90011A7406F080073099048A
:10379C00C299D211D006D005D000D0D0D082D0831F
:0337AC00D0E03238
:1017CE007879E6FE08E67C002400F547EC3EF54607
:1017DE00AF47FE123000501775240512418012419A
:1017EE0070AF47AE4612028CAF47AE4612200002D3
:0217FE00416642
:043000008E488F491E
:1030040090011AE07872666002C3227877E6FFF4D2
:10301400600DEF78756660077877E66002C3227802
:1030240078E66419600201AEFB7A0079777D0412B8
:103034003DD58E4A8F4B787BE6FE08E67C00240063
:10304400FFEC3EFEEF654B7003EE654A6002C3225F
:10305400787AE6FF18E6FEC39F40028002AF067846
:103064007AE6FDEEC39D400518E6FE8002AE0578C3
:1030740075E6FDC39F4005EDD39E4002C32278A9A7
:10308400E6FF7E00121FF6121FBF7C007D14121291
:10309400D28D4CE4F54DE54DC3954C500B7F647EC9
:1030A4000012414F054D80EED3227878E6FF640389
:1030B400600CEF64066007EF64106002C322787846
:1030C400E6FF6406703BD3E5499408E54894005054
:1030D40030787AE6FEC39402500990013EE030E075
:1030E40020C322EEC39404500990013EE030E11164
:1030F400C322787AE6B4080990013EE030E202C3C4
:1031040022E549640A4548703CEFB4030E121FBF20
:103114007C007D051212D27876A6057876E66401E5
:103124006002C322121FBF7C007D141212D28D4C88
:10313400E4F54DE54DC3954C500B7F647E00124180
:103144004F054D80EE7B007A00797790011AE024D8
:10315400FEFD123DD58E4A8F4B90011AE0FD247579
:10316400F8E6FE74762DF8E67C002400FFEC3EFEC3
:0B317400EFB54B06EEB54A02D322C3B4
:01317F00222D
:042000008E488F492E
:10200400E4F54EC20C7878E6FFB4061DE4F54E7490
:1020140077254EF8E6F599C2113011FD1241850578
:102024004EE54EC3940840E722EF64036002616604
:10203400787CE6F54C7877E6F54DF59912407F7893
:1020440078E6F54D3011FD12407CE54C25E0F54D68
:102054003011FD12407CE54EC3954C400261497E2F
:1020640000E549254EFFEE3548FEC3EF9464EE9437
:1020740000505DE54E2549FF7B007A00794AE4F57E
:1020840053121F084005E4F54AF54B7E00E5492547
:102094004EFFEE3548FEC3EF946EEE94004005E427
:1020A400F54D8004E54AF54D3011FD12407C7E006B
:1020B400E549254EFFEE3548FEC3EF946EEE9400DD
:1020C4004005754D018004E54BF54D3011FD61422D
:1020D4007E00E549254EFFEE3548FEEF64634E7001
:1020E40013F54D3011FD12407C90013EE0F54D306A
:1020F40011FD6142AF4E7E00E549254ECFEE3548D5
:10210400CF249CCF34FFFED3EF9407EE9400504AC3
:102114007E00E549254EFFEE3548FEEF25E0FFEE53
:1021240033FE74782FF58274003EF583E0F54D306C
:1021340011FD12407C7E00E549254EFFEE3548FE38
:10214400EF25E0FFEE33FE74782FF58274003EF540
:1021540083A3E0F54D3011FD6142AF4E7E00E549A9
:10216400254ECFEE3548CF249CCF34FFFEC3EF94E9
:1021740012EE9400504A7E00E549254EFFEE3548A4
:10218400FEEF25E0FFEE33FE74782FF58274003EF7
:10219400F583E0F54D3011FD12407C7E00E54925C4
:1021A4004EFFEE3548FEEF25E0FFEE33FE74782F48
:1021B400F58274003EF583A3E0F54D3011FD6142D4
:1021C4007E00E549254EFFEE3548FEC3EF9486EECA
:1021D4009400504EEF248AFFEE34FFFEEF25E0FF1B
:1021E400EE33FE741E2FF58274013EF583E0F54D47
:1021F4003011FD12407CAF4E7E00E549254ECFEEF6
:102204003548CF248ACF34FFFEEF25E0FFEE33FEBE
:10221400741F2FF58274013EF583E0F54D3011FDF6
:1022240061427E00E549254EFFEE3548FED3EF942A
:10223400ADEE9400501EE4F54D3011FD12407CE5E6
:102244004E2549246CF582E43400F583E0F54D30E5
:1022540011FD61427E00E549254EFFEE3548FEEF53
:1022640064AE4E7027F54D3011FD12407C7B007A30
:1022740000794AE4F5537F4D121F084006754A0061
:10228400754BFFE54BF54D3011FD61427E00E5498C
:10229400254EFFEE3548FED3EF94B6EE9400503F42
:1022A400EF25E0FFEE33FE74242FF58274FF3EF534
:1022B40083E0F54D3011FD12407C7E00E549254E4A
:1022C400FFEE3548FEEF25E0FFEE33FE74242FF5D4
:1022D4008274FF3EF583A3E0F54D3011FD805F7EEF
:1022E40000E549254EFFEE3548FED3EF94D6EE9433
:1022F40000503CE4F54D3011FD12407CE54E25497B
:102304002497FF7B007A00794AE4F553121F0840B2
:1023140005E4F54AF54BD3E54B940AE54A940040AD
:1023240005E4F54AF54BE54BF54D3011FD800FE41E
:10233400F54D3011FD12407C754D013011FD1240F8
:102344007C054E015AC20C3011FD7871E6F599C234
:10235400113011FD7873E6F599C21130110261FE56
:1023640080F97878E664107038F54E7477254EF865
:10237400E6F54DF599C2113011FDAF4D12408312AF
:102384004185054EE54EC3940640E07871E6F59923
:10239400C2113011FD7873E6F599C21120115B80EA
:1023A400FB7878E66419705218E6F54DF599C21178
:1023B4003011FDAF4D1240831241857878E6F54D1A
:1023C400F599C2113011FDAF4D1240831241857849
:1023D40075E6F54DF599C2113011FDAF4D124083EC
:1023E4001241857871E6F599C2113011FD7873E6D2
:0A23F400F599C2113011FD12418568
:0123FE0022BC
:04028C008E488F49C0
:10029000754E01E4F54F7878E664066002C14CC300
:1002A000E5499464E54894004002815E787AE694DA
:1002B000015021787CE6FD7C00E4FBFF123CD57800
:1002C0007BE6FD7C00E4FB7F01123CD590013EE023
:1002D00044018028787AE6D39403502A787CE6FD9E
:1002E0007C00E4FB7F02123CD5787BE6FD7C00E4D9
:1002F000FB7F03123CD590013EE04402F0FD7C0000
:10030000E4FB7F63C121787AE66408702E08E6FE7C
:1003100008E67C002400FDEC3EFCE4FB7F08123C78
:10032000D590013EE04404F0FD7C00E4FB7F6312C5
:100330003CD5787CE690013FF0C1C3787AE6B409F9
:100340001B08E6FE08E67C002400FDEC3EFCE4FB16
:100350007F09123CD5787CE6F51CC1C3787AE6FFAC
:10036000B4060A787CE6FD7C00E4FB807B787AE6C4
:10037000FFB40D1FC00708E6FE08E67C002400FD60
:10038000EC3EFCD007E4FB123CD5787CE69001956E
:10039000F0C1C3787AE6FFB40C1B787CE6FD7C00E4
:1003A000E4FB123CD5787CE6900197F06002C1C373
:1003B000752701C1C3787AE6FFB41012787CE6FD98
:1003C0007C00E4FB123CD5787CE6F54EC1C3787A1C
:1003D000E6640A70277876E664016002C1C3787C1F
:1003E000E6FD7C00E4FB7F06123CD5787CE6787560
:1003F000F67D067CEFE4FF123F7DC1C3E549640F43
:1004000045487019787AE6FF787CE6FD7C00E4FBCD
:10041000123CD5787CE6B40102801F8028E549644F
:10042000144548702B787AE6FF787CE6FD7C00E482
:10043000FB123CD5787CE6B4010B75878090011CDB
:100440007403F0C1C3E4F58790011C7406F0C1C3C6
:10045000787AE6FF787CE6FD7C00E4FBC121C3E509
:1004600049942CE54894014002C1C37879E6FE081E
:10047000E67C002400FFEC3ECF249CF549EF34FFDE
:10048000F548C3E5499412E5489400503808E6FE63
:1004900008E62400F54BEC3EF54AD3E54B94FFE526
:1004A0004A648094834002C1C3E54925E0FFE548E2
:1004B00033FE74402FF58274013EF583E54AF0A3C4
:1004C000E54BF0C1C3C3E549941AE54894005036A2
:1004D000E54924EEF54D787CE6FFC394064002C161
:1004E000C374B2254DF582E43400F583EFF0E54D99
:1004F000244EFF74B2254DF582E43400F583E0FD0F
:100500007C00E4FBC121D3E5499449E548940040CF
:1005100002A1AEC3E5499422E54894005002C1C34C
:10052000E54924DEFFE54834FFFE7C007D0512121C
:100530007D8F4D7B007A0079231240C74002C1C3F2
:10054000E54924DEFFE54834FFFE7C007D051212FC
:100550007DED4C70467A00796BAF4D1240B3E54D9E
:1005600025E025E024D2F582E43400F58312152538
:1005700000000000E54D25E025E02462F582E4342A
:1005800000F58312152500000000D21390011DE52F
:100590004DF07D017C007F08123EA0787CE6FF7460
:1005A000D02549F582E43400F583EFF0C1C3E54975
:1005B000644A45487021787CE6F523F54DD21290C7
:1005C000011BF0E54DFD7C00E4FB7F4D123CD59016
:1005D0000050741EF0C1C3C3E5499453E54894002C
:1005E0004044D3E5499472E54894005039E54924E4
:1005F000ADF54D787CE6FFC394064002C1C374B2EA
:10060000254DF582E43400F583EFF0E54D244EFFEF
:1006100074B2254DF582E43400F583E0FD7C00E4FE
:10062000FB123CD5C1C3E549646345486002C1C3C0
:10063000787CE6754A00F54BE4FBAD4BAC4A7F6332
:10064000123CD5787CE690013EF080777878E664BD
:10065000107070787CE6F97879E6FE08E67C002474
:1006600000F549EC3EF548749C2549F54974FF3581
:1006700048F548E4FDE9FFC3ED9FEC9400504412B7
:100680004185AF05EF25E0FB247EF8E6FE747F2B65
:10069000F8E67A002400F54BEA3EF54AE5492DFFDD
:1006A000E5483CFEEF25E0FFEE33FE74402FF58277
:1006B00074013EF583E54AF0A3E54BF00DBD000162
:1006C0000C80B2E54E647F70357F771207E4E4F565
:1006D0004C7B007A00794DE4F554AF4C123AE5506A
:1006E0000DE4254CFDE434EEFCAF4D123F7D054C8E
:1006F000E54CD3941040DAC2AF759F8080FEE54E82
:0A070000B4FF07C2AF759F8080FEB2
:01070A0022CC
:09417000787376FF787176FF2266
:07407C00854D99C211AF4D03
:104083007871E66FFF90265F937873667971F7EF27
:0540930090275F93F689
:014098002205
:083DD5008B4E8A4F89508D517D
:103DDD007552007553FF7DFFAF511551EF6026AB46
:103DED004E0550E550AA4F7002054F14F9121213EB
:103DFD006553FF90265F936D755200F553EF902735
:0A3E0D005F93FD80D3E553FEEDFF47
:013E17002288
:0240EF000000CF
:073BC70041006108011C0030
:103ED500E4F546751C01D20C7F0812070B500375DB
:103EE5004601751C02122F0A5003754602751C0304
:103EF500123E18EFD3940040028F4685461CE51C00
:0A3F0500FD7C00E4FB7F09023CD5BF
:102F0A001237AF900061E0FF139290EFA2E1929125
:102F1A00A2E292927FB1124000123BFCEF4E600295
:102F2A0080287F017E0012414F122FBC8E1A8F1B00
:102F3A00123F42400280137F017E0012414F122F3E
:102F4A00BC8E478F48123F424005124179C3227F07
:102F5A00017E0012414F122FBC8E498F4A124179CD
:102F6A00E51B2548FFE51A35475403F54B8F4C906E
:102F7A000061E0B4080EE54AB54C20E549B54B1BA3
:102F8A007D0F8010E54AB54C12E549B54B0D90000E
:102F9A0061E014FDAF48AE47122D86900061E0044F
:0B2FAA00F0E0D3940F40037408F0D354
:012FB50022F9
:103F9B008F461237AF7FB8124000123BFCEF4E60DA
:103FAB0005124179C3227F017E0012414FAF4612A9
:073FBB004000124179D322FE
:103E18001237AF7FB9124000123BFCEF4E6006121A
:103E280041797F00227F017E0012414F122FBC8F03
:103E380047123F427F017E0012414F122FBC8F482C
:103E4800E5476248124179E54870028003E4F54786
:023E5800AF4772
:013E5A002245
:103FC2008F461237AF7FBA124000123BFCEF4E60B1
:103FD20005124179C3227F017E0012414FAF461282
:073FE2004000124179D322D7
:1040DB00E51D6FFF90265F93651EF51DEF90275F23
:0340EB0093F51E2C
:0140EE0022AF
:1035B600751DFF751EFF1237AF7FB7124000123B15
:1035C600FCEF4E600280187F017E0012414F900092
:1035D60061E024F8FF124000123BFCEF4E6003024C
:1035E60041797F017E0012414F122FBC8F16123F88
:1035F600427F017E0012414F851646122FBC8F175F
:10360600123F427F017E0012414FE5176246122F9C
:10361600BC8F18123F427F017E0012414FE51862AF
:1036260046122FBC8F19123F427F017E0012414F76
:10363600E5196246122FBCAD07900061E024F8FF41
:10364600E434FFFEEF25E0FFEE33FE74002FF58233
:1036560074003EF583EDF0123F427F017E00124179
:103666004F900061E024F8FFE434FFFEEF25E0FF11
:10367600EE33FE74002FF5827400122FB6AD07905C
:103686000061E024F8FFE434FFFEEF25E0FFEE33AF
:10369600FE74012FF58274003EF583EDF0123F4271
:1036A6007F017E0012414F900061E024F8FFE43470
:1036B600FFFEEF25E0FFEE33FE74012FF582740066
:1036C600122FB6EF6246124179E5467029FF74164D
:1036D6002FF8E6B4010B74642567F567E43566F5E3
:1036E600660FBF02E9AF19AE18AD17AC16900061B0
:1036F600E0F54C1223FF900061E004F0E0D3940F54
:0537060040037408F00F
:01370B00229B
:02070B008F4716
:10070D0078487C007D007BFF7A4079EF7E007F1476
:10071D001211EDC290C291C2921237AF300C047F0C
:10072D00B18005200C057FB21240007F017E0012C2
:10073D00414F123BFCEF4E600280167F017E00128E
:10074D00414F122FBC8E488F49755C01123F4240BC
:10075D0005124179C3227F017E0012414FE55C13E2
:10076D009290E55CA2E19291A2E29292122FBCE5E9
:10077D005C25E02448F8A60608A607055CE55CD3D1
:10078D00940940C8124179E549254BCFE548354AD2
:10079D00CF254DCF354CCF254FCF354ECF2551CF12
:1007AD003550CF2553CF3552CF2555CF3554CF2585
:1007BD0057CF3556CF2559CF35585403FEE55BB588
:1007CD000713E55AB5060E7B007A00794885476117
:0607DD007D08122BD8D3A9
:0107E30022F3
:1037AF00C2967F017E0012414FD297D2967F027E42
:1037BF000012414FC2977F057E0012414FC2967F84
:1037CF00027E0012414FE51CB402028005E51CB4D5
:1037DF00031DD297D2967F027E0012414FC2977F70
:1037EF00057E0012414FC2967F027E0012414F228A
:103F4200E4FFFE20970D0FBF00010EEF64644E7078
:103F5200F2C322D2977F017E0012414FD296C297BE
:0C3F62007F017E0012414FD297C296D31F
:013F6E002230
:02400000AD070A
:104002007B08ED339297D2967F017E0012414FC218
:0E401200967F017E0012414FED25E0FDDBE4BC
:01402000227D
:062FB6003EF583E06246D7
:102FBC00E4FBFAE51CB403047D0880027D0AE4F905
:102FCC00E9C39D5028D2967F017E0012414FD297C3
:102FDC00EB25E0FFEA33FEA297E433FBEEFAEF4B6E
:102FEC00FBC2967F017E0012414F0980D3AE02AF27
:012FFC0003D1
:012FFD0022B1
:07417900C297D296D29722F3
:103BFC00E4F55DF55EE51C64017018D297D296FA77
:103C0C00FB20970280460BBB00010AEB640A4A704A
:103C1C00F0804AE51C6402701DFAFB20970BD296CB
:103C2C007F017E0012414F80230BBB00010AEB6425
:103C3C00324A70E78027E51C64037027FAFBD297A1
:103C4C0020970FD2967F017E0012414FC296E4FE60
:103C5C00FF220BBB00010AEB64324A70E1C2967E74
:033C6C00007F01D5
:013C6F002232
:062D86008E4D8F4E8D4FB3
:102D8C00E54F25E02440F582E43401F583E0FEA311
:102D9C00E0FFC3E54E9FFFE54D9EFE124139D3EF98
:102DAC009464EE6480948040467492254FF582E4DE
:102DBC003400F583E004F07492254FF582E434007E
:102DCC00F583E0D3648094825002C1737492254FD2
:102DDC00F582E43400F583E4F0E54F25E02440F57A
:102DEC0082E43401F583E54DF0A3E54EF080787470
:102DFC0092254FF582E43400F583E4F0E54F25E0AD
:102E0C002440F582E43401F583E0FEA3E0FFE4FC0A
:102E1C00FD7B02FAF9F81213D8C004C005C006C035
:102E2C0007AE4DAF4EE4FCFD7B08FAF9F81213D84F
:102E3C00D003D002D001D000EB2FFFEA3EFEE93DDB
:102E4C00FDE83CFCE47B0AFAF9F81214638F538E0C
:102E5C00528D518C50E54F25E02440F582E434012D
:102E6C00F583EEF0A3EFF0E54F25E02440F582E486
:102E7C003401F583E0FCA3E0FD74AA254FF582E450
:102E8C003400F583E0FF7B807A00123180E54F251A
:102E9C00E02400F582E43400F583EEF0A3EFF0E5D6
:102EAC004F25E02440F582E43401F583E0FEA3E0F5
:102EBC00D39400EE94044013E54F25E02440F582B2
:102ECC00E43401F5837404F0A3E4F0E54F25E02429
:102EDC0040F582E43401F583E0FEA3E0FFE4FCFD61
:102EEC007B607AEAF9F8C31215035011E54F25E01F
:0D2EFC002440F582E43401F583E4F0A3F0F6
:012F090022A5
:0823FF008F4B8E4A8D498C487A
:10240700E54C24F8F54D900050E0D394004003E0EC
:1024170014F07B007A007923AF4D1240C740028148
:10242700D6900050E060028055E54D25E025E02478
:1024370062F582E43400F583E0F8A3E0F9A3E0FA5B
:10244700A3E0FBC3E54B9BF552E54A9AF551E549F5
:1024570099F550E54898F54F7F007EF07DFF7CFFAA
:10246700AB52AA51A950F8D31215035002A198E410
:10247700FF7E10FDFCA84F1215034002A198E54C02
:1024870025E025E024B2F582E43400F583E0FCA3DF
:10249700E0FDA3E0FEA3E0254BFFEE354AFEED3558
:1024A70049FDEC3548FCE54D25E025E0241EF58285
:1024B700E43401F583121519AF4BAE4AAD49AC4868
:1024C700E54D25E025E02462F582E43400A19390F0
:1024D7000050E06047AF4BAE4AAD49AC48E54D25EB
:1024E700E025E02462F582E43400F58312151974BF
:1024F700B2254DF582E43400F583E0FFAC4AAD4BDD
:102507007B807A00123180EE3395E0FDFCE54D25A6
:10251700E025E0241EF582E434018070E54D25E0D6
:1025270025E02462F582E43400F583A3A3E0FEA34B
:10253700E0FFC3E54B9FFFE54A9EFE1241398F4EF0
:10254700E54EC394FF504AAF4BAE4AAD49AC48E5A0
:102557004D25E025E02462F582E43400F583121569
:102567001974B2254DF582E43400F583E0FFAC4AD7
:10257700AD4B7B807A00123180EE3395E0FDFCE5B0
:102587004D25E025E0241EF582E43401F58312157C
:1025970019900050E06002804CE54D25E0FDE433E2
:1025A700FC74002DF58274003CF583E0FE74012D68
:1025B700F58274003CF583E07C002400FFEC3EFECE
:1025C700E54D25E02451F582E43400F583E0FCA3D2
:1025D700E0FDC3EF9DFFEE9CFE1241398F4EE54EA5
:1025E700C394FF5072E54D25E0FDE433FC74002DE4
:1025F700F58274003CF583E0FE74012DF5827400CA
:102607003CF583E07C002400FFEC3EFEE54D25E031
:102617002451F582E43400F583EEF0A3EFF0E54DA5
:1026270025E0FDE433FC74002DF58274003CF5834E
:10263700E0FE74012DF58274003CF583E07C0024F4
:1026470000FFEC3EFEE54D25E02482F582E43400F0
:07265700F583EEF0A3EFF0A4
:01265E002259
:082BD8008B5D8A5E895F8D6050
:102BE000E4F564E564C395604002A185AB5DAA5E2F
:102BF000A95FE5640475F002A4F58285F0831213E1
:102C000049FFAEF0E564256125E02440F582E43417
:102C100001F583E0FCA3E0FDC3EF9DF563EE9CF5B9
:102C200062C3E5639464E56264809480500DC3E5FB
:102C300063949CE5626480947F5023E5642561FD84
:102C400025E02440F582E43401F583EEF0A3EFF0B3
:102C500074922DF582E43400F583E4F08059AB5D85
:102C6000AA5EA95FE5640475F002A4F58285F0838D
:102C7000121349FFAEF0E5642561FD25E02440F51F
:102C800082E43401F583E0FAA3E0FBC39FEA9E509F
:102C90000F74922DF582E43400F583E004F0801780
:102CA000D3EB9FEA9E4010E56425612492F582E40F
:102CB0003400F583E014F0E56425612492F582E4A4
:102CC0003400F583E0FFD36480948A500AC3EF6434
:102CD0008094764002A181D3E5639414E562648018
:102CE0009480500DC3E56394ECE5626480947F505A
:102CF0001FAE62AF637C007D051212D2E5642561D0
:102D000025E02440F582E43401F583EE8FF0805F06
:102D1000AB5DAA5EA95FE5640475F002A4F5828547
:102D2000F083121349FFAEF0E5642561FD25E02430
:102D300040F582E43401F583E0FAA3E0FBC39FEAA7
:102D40009E5012ED25E02440F582E43401F583E441
:102D500075F001801AD3EB9FEA9E4016E564256169
:102D600025E02440F582E43401F58374FFF5F01288
:102D70001308E56425612492F582E43400F583E4C8
:052D8000F0056461E3B1
:012D8500222B
:103F0F000205050506060606070707080809090A38
:103F1F000B0C0C0D0E10121315171B1E252A2F3606
:103F2F003A3B37312C26231E1D1818151513111166
:033F3F00100F0F51
:103BCE004101BA004101B700017000C1154201B8B0
:023BDE00012CB8
:10080000E4F548F549200A3DD293A29033FDA29128
:10081000E433FBA292E433FA9001BAE0FF13929022
:10082000EFA2E19291A2E29292C2B37FF47E011212
:10083000414FD2B3ED24FF9290EB24FF9291EA2432
:10084000FF9292C2939001BAE00475F00D84E5F036
:10085000F0900197E0FF60022159300A6B200202FC
:1008600021599001B7E0640C705CE5700475F00DDF
:100870008485F070C202D208301528E57025E02486
:1008800040F582E43401F5837403F0A374E8F0E5E5
:1008900070B40702C215E49001B7F0E52760271590
:1008A000272153E57025E02440F582E43401F583E7
:1008B000E4F0A3F0E570B40702D215E49001B7F0BC
:1008C000E52760021527215320020221599001BA21
:1008D000E0FE9001B830E012E0FCA3E0FDC374E854
:1008E0009DF54774039CF5468007E0F546A3E0F5C7
:1008F00047C374079E25E02440F582E43401F58364
:10090000E546F0A3E547F09001B7E064207044C2EB
:1009100002D20830151B9001B9E02464F09001B8B0
:10092000E03400F0E0B40320A3E0B4E81BC215807B
:10093000179001B9E0249CF09001B8E034FFF0E09A
:100940007002A3E07002D215E49001B7F0E52760D1
:100950000215279001B7E004F0200A02615E9001C1
:10096000BAE0FE24F76071147002413A147002413B
:100970009C14700241FE24046002615E74AA2EF889
:10098000E6FE700EEF600B300004C290615ED29004
:10099000615EEEB40111900197E0600B300004D26B
:1009A00090615EC290615E9001BAE025E02440F55E
:1009B00082E43401F583E0FEA3E0D394F4EE9401E5
:1009C000400B300004D290615EC290615E30000442
:1009D000C290615ED290615E9001BAE024AAF8E60E
:1009E000FF7011900197E0600B300004C291615ECE
:1009F000D291615EEFB40111900197E0600B30007D
:100A000004D291615EC291615E9001BAE025E0245A
:100A100040F582E43401F583E0FEA3E0D394F4EEE4
:100A20009401400B300004D291615EC291615E304E
:100A30000004C291615ED291615E9001BAE024AA85
:100A4000F8E6FF7011900197E0600B300004C2924D
:100A5000615ED292615EEFB40111900197E0600B8C
:100A6000300004D292615EC292615E9001BAE025CC
:100A7000E02440F582E43401F583E0FEA3E0D39462
:100A8000F4EE9401400B300004D292615EC2926198
:100A90005E300004C292615ED292615E9001BAE063
:100AA00024AAF8E6FF7011900197E0600B30000473
:100AB000C293615ED293615EEFB40111900197E041
:100AC000600B300004D293615EC293615E9001BA04
:100AD000E025E02440F582E43401F583E0FEA3E064
:100AE000D394F4EE9401400B300004D293806FC293
:100AF00093806B300004C2938064D2938060900135
:100B0000BAE024AAF8E6FF7011900197E0600B307C
:100B10000004C2DB8048D2DB8044EFB401119001B5
:100B200097E0600B300004D2DB8033C2DB802F9073
:100B300001BAE025E02440F582E43401F583E0FECB
:100B4000A3E0D394F4EE9401400B300004D2DB8098
:100B50000DC2DB8009300004C2DB8002D2DB200A38
:100B600002C1529001BAE0FFB408004002C1B79040
:100B70000B7525E073618561DC8136819081EAA186
:100B800044A19EA1F874AA2FF8E6FF700F90019778
:100B9000E06009300003C2A022D2A022EFB4010F0E
:100BA000900197E06009300003D2A022C2A02290F9
:100BB00001BAE025E02440F582E43401F583E0FE4B
:100BC000A3E0D394F4EE94014009300003D2A022B4
:100BD000C2A022300003C2A022D2A0229001BAE01B
:100BE00024AAF8E6FF700F900197E0600930000337
:100BF000C2A122D2A122EFB4010F900197E06009B7
:100C0000300003D2A122C2A1229001BAE025E02443
:100C100040F582E43401F583E0FEA3E0D394F4EEE2
:100C200094014009300003D2A122C2A12230000366
:100C3000C2A122D2A1229001BAE024AAF8E6FF7054
:100C40000F900197E06009300003C2A222D2A222D5
:100C5000EFB4010F900197E06009300003D2A222A7
:100C6000C2A2229001BAE025E02440F582E43401DA
:100C7000F583E0FEA3E0D394F4EE94014009300044
:100C800003D2A222C2A222300003C2A222D2A222F6
:100C90009001BAE024AAF8E6FF700F900197E06097
:100CA00009300003C2A322D2A322EFB4010F9001A6
:100CB00097E06009300003D2A322C2A3229001BAB8
:100CC000E025E02440F582E43401F583E0FEA3E072
:100CD000D394F4EE94014009300003D2A322C2A3BE
:100CE00022300003C2A322D2A3229001BAE024AA98
:100CF000F8E6FF700F900197E06009300003C2A48E
:100D000022D2A422EFB4010F900197E060093000D5
:100D100003D2A422C2A4229001BAE025E02440F527
:100D200082E43401F583E0FEA3E0D394F4EE940171
:100D30004009300003D2A422C2A422300003C2A47E
:100D400022D2A4229001BAE024AAF8E6FF700F9004
:100D50000197E06009300003C2A522D2A522EFB4BA
:100D6000010F900197E06009300003D2A522C2A5CF
:100D7000229001BAE025E02440F582E43401F583B5
:100D8000E0FEA3E0D394F4EE94014009300003D2D6
:100D9000A522C2A522300003C2A522D2A52290011D
:100DA000BAE024AAF8E6FF700F900197E0600930DE
:100DB0000003C2A622D2A622EFB4010F900197E051
:100DC0006009300003D2A622C2A6229001BAE02513
:100DD000E02440F582E43401F583E0FEA3E0D394FF
:100DE000F4EE94014009300003D2A622C2A62230BC
:100DF0000003C2A622D2A6229001BAE024AAF8E6F5
:100E0000FF700F900197E06009300003C2A722D263
:100E1000A722EFB4010F900197E06009300003D2E0
:100E2000A722C2A7229001BAE025E02440F582E47F
:100E30003401F583E0FEA3E0D394F4EE940140097D
:100E4000300003D2A722C2A722300003C2A722D2B9
:100E5000A7229001BAE0FFC374079F24AAF8E6FF17
:100E6000700A900197E06004E4F5A722EFB4010C4A
:100E7000900197E060067FFF7E0380369001BAE024
:100E8000FFC374079F25E02440F582E43401F58315
:100E9000E0FEA3E0FF900195E0FD7C00EF2DFFEC6C
:100EA0003ECF2480CF34FFFEC3648094805003E49F
:070EB000FEFF123A4E8FA76E
:010EB7002218
:043A4E008E4A8F4BC2
:103A5200E4F54C903F0F93754D00F54ED3E54E952E
:103A62004BE54D954A4004E4FFFE22054CAF4CEF76
:103A72003395E0FE740F2FF582743F3EF583E49395
:103A8200F9254EF54EE4354DF54DD3E54E954BE512
:103A92004D954A4046E54E954BFFE54D954AFEE968
:103AA200C39FFBE49E7C007D0AAF03FE12126BE90A
:103AB200FD1212D27C007D0512126B7D0A1212D207
:103AC200AA06AB07AF4CEF3395E0FE7C007D0512F2
:103AD200126BEF2BFBEE3AAF03FE22E54C708C7FAC
:023AE200FFFEE5
:013AE40022BF
:0301000014000EDA
:10409900C0D1CEBBA183674F3D2D9B19273D5366E8
:0A40A900717065554333261C154164
:023BE000C1968C
:04345C008E548F55A6
:103460007B0EEB30160E3395E0FE74A4240EF5822D
:103470007440800CFF3395E0FE74992FF582744000
:103480003EF583E493FF9001B5E4F0A3EFF0D39011
:1034900001B6E095559001B5E095544004EBFFA1CD
:1034A0009A1BEBFF3395E0FE30160974A42FF582CA
:1034B0007440800774992FF58274403EF583E4933D
:1034C000FF9001B6E02FF09001B5E03400F09001DC
:1034D000B5E0FEA3E0FFD39555EE95545002A192BE
:1034E000EF9555FFEE9554FE7C007D6412126B90B3
:1034F00001B3EEF0A3EFF09001B3E0FEA3E0FFEB29
:10350000FD3395E0FC30160974A42DF582744080DB
:103510000774992DF58274403CF583E493FD7C009B
:103520001212D29001B3EEF0A3EFF0C3EB648094DB
:1035300084EBFF40253395E0FEEF24FCFFEE34FFE3
:10354000FE7C007D6412126B9001B4E02FF09001BC
:10355000B3E03EF0E0547FF080533395E0FE7C0012
:103560007D6412126B9001B4E02FF09001B3E03E45
:10357000F0E0FEA3E0FFC374909FFF74019EFE90F5
:1035800001B3F0A3EFF0EE44809001B3F0A3EFF0AD
:10359000801BEB600281A1AF03EF3395E0FE7C005E
:1035A0007D6412126B9001B3EEF0A3EFF09001B3C3
:0535B000E0FEA3E0FFB6
:0135B50022F3
:103180009001ACEFF0A3ECF0A3EDF0A3EAF0A3EB19
:10319000F0EF701E9001AFE0FEA3E0FF9001AEE003
:1031A0002FFF9001ADE03ECF2480CF34FF9001B1DE
:1031B00041ED9001ACE0FF64016005EF6402707CBA
:1031C0009001ADE0FEA3E0FF12345C9001AAEEF0A6
:1031D000A3EFF0EE9001AA30E712E0547FFEA3E0E7
:1031E000FFC3E49FFFE49E9001B18008E0FFA3E0ED
:1031F0009001B1CFF0A3EFF09001ACE0B4022290C7
:1032000001B1E0FEA3E0FF7C007D0912126B7D0599
:103210001212D2EF2440FFEE34019001B1F0A3EF7F
:10322000F09001AFE0FEA3E0FF9001B2E02FFF902D
:1032300001B1E03ECF2480CF34FF41ED9001ACE0FE
:10324000B40328A3E0FCA3E0FDEC1210637B007A3A
:10325000C0797F7844120FC1E4FBFA79C878421232
:103260000EB812109C9001B1EE41ED9001ACE0FF60
:1032700064046005EF640570789001ADE0FCA3E0A4
:10328000FDEC1210637B007AC0797F7844120FC185
:10329000E4FBFA79487842120EB812109C9001AA09
:1032A000EEF0A3EFF0D39418EE648094805012A354
:1032B000E0FFB40504D20C802BEFB40427C20C80CD
:1032C00023C39001ABE0941A9001AAE0648094803B
:1032D00040129001ACE0FFB40504C20C8006EFB4CC
:1032E0000402D20CA20CE4FF339001B1CFF0A3EFA3
:0932F000F09001B1E0FEA3E0FF43
:0132F90022B2
:103BE2004401A60200020048019E006800690066C6
:093BF200006744019A0002000280
:0E3F6F00855783E4939001B1FFF0AC59AD5A31
:103F7D00AB07C2AF75F65575F6AA75F65543BF0476
:0E3F8D008CF48DF58BF675F780D2AF7F002295
:1007E400C2AF75F65575F6AA75F65543BF04EF25E5
:0C07F400E0F5F4E4F5F575F782D2AF22D1
:0B415A008F828E83E4931212597F01C4
:014165002237
:0C402100E54775F002A4240CF9E4FAFB5A
:10402D0012131EF58285F083E4932402FFE4338F8F
:04403D00F0021381F9
:023E5B00A907B5
:103E5D00E925E0249AF582E43401F583A3E0F556D3
:103E6D00E925E0240CF8E6FE08E6FFE5562402FD00
:103E7D00E433FCE925E02410F8E6FA08E6C39DFDDD
:0D3E8D00EA9CFCC3EF9DEE9C4002D322C3D3
:013E9A002205
:10412700E4F546AF461215560546E546C3940240E8
:01413700F295
:014138002264
:021556008F47BD
:10155800EF25E024A6F582E43401F583E0F54AA3FB
:10156800E0F54BEF25E025E0249EF582E43401F513
:1015780083A3E0F548EF25E025E024A0F582E434D4
:1015880001F583A3E0F549E54825E0F54C754D00E4
:10159800E54925E0754EFFF54F755000854D82856C
:1015A8004C83E49364556002C1FCAB4EAA4FA9502A
:1015B80012121364556002C1FCE54D2401FFE435A5
:1015C8004CFEE54725E0240CF8A60608A607E547E3
:1015D80025E0240CF8E6FE08E6F5828E83E493F411
:1015E8006020E54725E0240CF8E6FE08E6AA06C3D5
:1015F800854F838550829582EA9583500512402154
:1016080080CCE54725E0240CF8E6FE08E6C3954DB6
:10161800F552EE954CF551E5502401F9E4354FFEAD
:10162800AF01E54725E0240CF8A60608A607E5471C
:1016380025E0240CF8E6FE08E6F5828E83E493F4B0
:101648006030AB4EE550254BF9E54F354AFAC003FB
:101658008A838982E54725E0240CF8E6FE08E6AA95
:1016680006F9C3D0E0E99582EA9583500512402136
:1016780080BCE54725E0240CF8E6FE08E6AB4EAA58
:101688004FA950AC02AD01C39DFFEE9CFED3EF9570
:1016980052EE95515032AE02AF01EF2401FFE43E05
:1016A800FEE54725E02408F8A60608A607741425D1
:1016B80047F8A648AE4CAF4DAD07AC06E4FF123F65
:1016C8007DEF7002E17DC322E54D2401FFE4354C36
:1016D800FEE54725E02408F8A60608A607741425A1
:1016E80047F8A649AC4FAD50E4FF123F7DEF7002BA
:1016F800E17DC322854D82854C83E493B4551EE574
:101708004D2401FFE4354CFEE54725E02408F8A602
:101718000608A60774142547F8A6498058AB4EAAB0
:101728004FA950121213B45520AE02AF01EF240195
:10173800FFE43EFEE54725E02408F8A60608A607CC
:1017480074142547F8A648802CAE4CAF4DAD07ACB5
:1017580006ED2401FFE43CFEE54725E02408F8A651
:101768000608A60774142547F8A6497F55123F7D39
:10177800EF6002C322E54725E02408F8E6FE08E604
:10178800FFE54725E0240CF8A60608A607E5472547
:10179800E02408F8E6FE08E6254BFFE54A3EFEE5AC
:1017A8004725E02410F8A60608A607E54725E02403
:1017B8000CF8E6FE08E6F5828E83E493F4600512E1
:0517C800402180E7D381
:0117CD0022F9
:02285F008F5692
:10286100EF25E02408F8E6FE08E68E57F5587414C3
:102871002FF8E625E0F559755A00E55625E024A61E
:10288100F582E43401F583E0FFA3E09001B2CFF0DB
:10289100A3EFF0E49001AEF0E55625E024A6F58221
:1028A100E43401F583E0C313FF9001AEE0C39FE47C
:1028B1009400501512418574142556F8E6FFE02F57
:1028C100FF1207E4E004F080CF9001B3E02558FF48
:1028D1009001B2E03557CF24FFF55CEF34FFF55B93
:1028E100055AE55A70020559855882855783E49344
:1028F100F47002218FC3E558955CE557955B400262
:10290100218F124185855882855783740193FF6019
:1029110072F4606FE4939001AF123F77EF60037F31
:102921000122055AE55A700205590558E558700209
:102931000557F582123F6FEF60037F0122055AE5CB
:102941005A700205590558E55870020557E490017F
:10295100AEF09001AFE0FF9001AEE0C39F508985DA
:102961005882123F6FEF60037F0122055AE55A70CA
:102971000205590558E558700205579001AEE0046B
:10298100F080CF7B007A00795712402D01E9E5569E
:1029910025E0240CF8A65908A65AE55625E0240896
:1029A100F8E6FEEEC3139001B0F0FD74142556F85D
:1029B100E625E0FEE55625E02408F8A6060876009F
:1029C10074142556F8A605E55625E02408F8E6FE18
:1029D10008E6FF9001B3E02FFF9001B2E03EFEE573
:1029E1005625E02410F8A60608A607E55625E0249A
:1029F10008F8E6FC08E6FD7F55123F7DEF60037F96
:102A0100012274142556F8E67D0025E0FCE4FF124E
:102A11003F7DEF60037F0122E55625E02408F80899
:082A210006E6187001067F00B3
:012A2900228A
:083800008F568B578A58895935
:10380800E4F55EF55FE55A25E0249AF582E4340193
:10381800F583A3E0F560E55A25E02408F8E6FE08FC
:10382800E68E5BF55C0556E55A25E0240CF8E6FEC5
:1038380008E6FFE5602401FDE433FCE55A25E024B1
:1038480010F8E6FA08E6C39DFDEA9CFCD3EF9DEE6E
:103858009C400122855C82855B83740193FE6556DA
:103868006010E493F4600B7B007A00795B12402DC2
:1038780080E2EEB5560BE55C2401F55FE4355BF5B7
:103888005EE55A25E0240CF8E6FE08E6FDAC06AF36
:1038980060123F7DEF6002C322E55A25E0240CF850
:1038A80008740226F618E436F6E4F55DE55DC3957E
:1038B800605030E55A25E0240CF8E6FE08E6255D60
:1038C800FFE43EFEAD07FCAB57AA58A959855D82B7
:1038D80075830012122CFF123F7DEF6002C3220590
:1038E8005D80C9AF607E00E55A25E0240CF808EF3A
:1038F80026F618EE36F6E55A25E0240CF8E6FC081C
:10390800E6FDEF2401FFEE33FEC3ED9FFFEC9EFEC4
:10391800AD07FCAF56123F7DEF6002C322E55F455D
:103928005E6012AE5EAF5FAD07AC06E4FF123F7D8E
:06393800EF6002C322D380
:01393E002266
:081F08008F4F8B508A51895262
:101F1000E55325E02408F8E6FE08E68E54F555E47E
:101F2000F556F557054F855582855483E493F46043
:101F300049E55325E02410F8E6FC08E6FDC3E55525
:101F40009DE5549C5034740193654F7022E55745CC
:101F5000566016E5572401FFE43556FEAD07FCE454
:101F6000FF123F7DEF6002C3228554568555577B93
:101F7000007A00795412402D80ACE5574556603DFB
:101F8000855782855683740293FFAB50AA51A9529C
:101F9000E48FF01213B9AB50AA51A95212131E7557
:101FA000F0001213B9855782855683740393FFABF3
:0E1FB00050AA51A952E48FF0121381D322C31C
:011FBE002200
:083AE5008F508B518A52895366
:103AED00E55425E02408F8E6FE08E68E55F556E483
:103AFD00F557F5580550855682855583E493F46046
:103B0D0049E55425E02410F8E6FC08E6FDC3E5562A
:103B1D009DE5559C503474019365507022E55845D0
:103B2D00576016E5582401FFE43557FEAD07FCE458
:103B3D00FF123F7DEF6002C3228555578556587B96
:103B4D00007A00795512402D80ACE5584557601428
:103B5D00855882855783740393AB51AA52A953128A
:053B6D001259D322C330
:013B72002230
:043CD5008F508B5130
:103CD900E4F552EDF554ECF553124185AF51123E1E
:103CE9005B5022E552C3940A500CAF5112285FEF82
:103CF9006004055280ED7F057E0012414FE552C3F5
:103D0900940A400122E552C3940A50147B007A00B8
:103D1900795385515AAF501238004004055280E555
:093D2900E552C3940A400122D3C3
:013D3200226E
:100EB800EC4D6011E8497017ED33EC3304600DE434
:100EC800FCFFFEFD22E933E8330470F80211081232
:100ED80010D358046009E4CC248150062850090234
:100EE800111228400302110FC0E0EB4A7044B98088
:100EF80006D0E0FB0210FEEF4E701CBD8008EBFF31
:100F0800EAFEE9FD80EBE98DF0A4FEE5F0020FA111
:100F1800E9CDF9EAFEEBFFEF89F0A4FCE5F0CE8914
:100F2800F0A42EFFE435F0CD89F0A42DFEE435F0D1
:100F38008067EF4E7005BD80D780C3EF8BF0A4ACFF
:100F4800F0EE8BF0A42CFCE435F0F8EF8AF0A42C3A
:100F5800E5F038FCE433CB8DF0A42CFCE5F03BF84D
:100F6800EE8AF0A42CFCE5F038F8E433CF89F0A43D
:100F78002CFCE5F038CF3400CE89F0A42FFFE5F043
:100F88003EFEE433C98DF0A42EFEE5F039CD8AF09B
:100F9800A42FFFE5F03EFEE43DFD33D0E0FB500713
:100FA8000BBB000F021112EC2CFCEF33FFEE33FEEB
:060FB800ED33FD0210EA1A
:100FBE00021112EC5D046005E85904700302110879
:100FCE001210D3580460F6EC4860F2EC7004FDFE8B
:100FDE00FF22C860DB2481C85009C3986002500606
:100FEE0002110F9850CAF582E9294B4A7005AB825F
:100FFE000210FE75F0007C1A7880C3EF9BEE9AED1E
:10100E0099400DC3EF9BFFEE9AFEED99FDE842F07D
:10101E00DC23ACF0D0E0FFD0E0FED0E0FDAB8220D0
:10102E00E7101BEB60BAEC2CFCEF33FFEE33FEED5A
:10103E0033FD0210EAE803F830E705C0F075F00062
:10104E00EF2FFFEE33FEED33FD40B830E7C280AA3E
:10105E0075F020800E75F010800575F0087D007E0D
:10106E00007F003392D530D5031214F5EC334010C7
:10107E00EF33FFEE33FEED33FDEC33FCD5F0ED2216
:0E108E00E5F0247EA2D513CC92E7CDCEFF2252
:10109C00EDD2E7CD33EC3392D524814006E4FFFE4C
:1010AC00FDFC22FCE4CFCECDCC24E0501174FF80AB
:1010BC00EDC3CC13CCCD13CDCE13CECF13CF047048
:0710CC00F030D5DE0214F53F
:1010D300E9D2E7C933E833F892D5EDD2E7CD33EC63
:0710E30033FC5002B2D522DC
:1010EA00EC30E7100FBF000C0EBE00080DBD000467
:1010FA000BEB6014A2D5EB13FCED92E7FD2274FF13
:10110A00FCFDFEFF22E480F8A2D574FF13FC7D806B
:03111A00E480EF7F
:03000000020200F9
:0C020000787FE4F6D8FD7581C902024742
:10111D00E709F608DFFA8046E709F208DFFA803EB4
:10112D0088828C83E709F0A3DFFA8032E309F608A1
:10113D00DFFA8078E309F208DFFA807088828C8309
:10114D00E309F0A3DFFA806489828A83E0A3F608BD
:10115D00DFFA805889828A83E0A3F208DFFA804C97
:10116D0080D280FA80C680D4806980F2803380106E
:10117D0080A680EA809A80A880DA80E280CA8033D7
:10118D0089828A83ECFAE493A3C8C582C8CCC5834F
:10119D00CCF0A3C8C582C8CCC583CCDFE9DEE7801F
:1011AD000D89828A83E493A3F608DFF9ECFAA9F09E
:1011BD00EDFB2289828A83ECFAE0A3C8C582C8CCF4
:1011CD00C583CCF0A3C8C582C8CCC583CCDFEADE0D
:1011DD00E880DB89828A83E493A3F208DFF980CC6F
:1011ED0088F0EF60010E4E60C388F0ED2402B40468
:1011FD000050B9F582EB2402B4040050AF2323450F
:06120D00822390116D73B5
:10121300BB010689828A83E0225002E722BBFE02D9
:09122300E32289828A83E493220C
:10122C00BB010CE58229F582E5833AF583E0225077
:10123C0006E92582F8E622BBFE06E92582F8E222C1
:0D124C00E58229F582E5833AF583E49322DB
:10125900BB010689828A83F0225002F722BBFE0174
:02126900F3226E
:10126B00EF8DF0A4A8F0CF8CF0A428CE8DF0A42E97
:02127B00FE2251
:10127D00BC000BBE0029EF8DF084FFADF022E4CC55
:10128D00F875F008EF2FFFEE33FEEC33FCEE9DEC1E
:10129D00984005FCEE9DFE0FD5F0E9E4CEFD22ED64
:1012AD00F8F5F0EE8420D21CFEADF075F008EF2FAE
:1012BD00FFED33FD4007985006D5F0F222C398FD9F
:0512CD000FD5F0EA223C
:1012D200C2D5EC30E709B2D5E4C39DFDE49CFCEE37
:1012E20030E715B2D5E4C39FFFE49EFE12127DC320
:1012F200E49DFDE49CFC800312127D30D507C3E41B
:061302009FFFE49EFE22A5
:10130800C5F0F8A3E028F0C5F0F8E5821582700270
:061318001583E038F0220D
:10131E00BB010A89828A83E0F5F0A3E0225006879A
:10132E00F009E71922BBFE07E3F5F009E31922895C
:0B133E00828A83E493F5F0740193228F
:10134900BB0110E58229F582E5833AF583E0F5F0E2
:10135900A3E0225009E92582F886F008E622BBFEBF
:101369000AE92582F8E2F5F008E222E5832AF58305
:08137900E993F5F0A3E99322CA
:10138100BB010789828A83021308500B09C5F02724
:10139100F7C5F01937F722BBFE0D09F8E325F0F385
:1013A100C5F019E338F322F889828A837401932501
:0813B100F0C5F0F8E4933822C6
:1013B900BB010A89828A83F0E5F0A3F0225006F77F
:0F13C90009A7F01922BBFE06F3E5F009F319227C
:1013D800E88FF0A4CC8BF0A42CFCE98EF0A42CFCB4
:1013E8008AF0EDA42CFCEA8EF0A4CDA8F08BF0A432
:1013F8002DCC3825F0FDE98FF0A42CCD35F0FCEB91
:101408008EF0A4FEA9F0EB8FF0A4CFC5F02ECD3955
:0F141800FEE43CFCEAA42DCE35F0FDE43CFC22C2
:1014270075F008758200EF2FFFEE33FECD33CDCC7C
:1014370033CCC58233C5829BED9AEC99E5829840FF
:101447000CF582EE9BFEED9AFDEC99FC0FD5F0D6DC
:10145700E4CEFBE4CDFAE4CCF9A88222B800C1B906
:101467000059BA002DEC8BF084CFCECDFCE5F0CB44
:10147700F97818EF2FFFEE33FEED33FDEC33FCEB7D
:1014870033FB10D703994004EB99FB0FD8E5E4F938
:10149700FA227818EF2FFFEE33FEED33FDEC33FC25
:1014A700C933C910D7059BE99A4007EC9BFCE99A19
:1014B700F90FD8E0E4C9FAE4CCFB2275F010EF2F5E
:1014C700FFEE33FEED33FDCC33CCC833C810D7075E
:1014D7009BEC9AE899400AED9BFDEC9AFCE899F899
:0E14E7000FD5F0DAE4CDFBE4CCFAE4C8F9222C
:0E14F500C3E49FFFE49EFEE49DFDE49CFC2208
:10150300EB9FF5F0EA9E42F0E99D42F0EC6480C85F
:0615130064809845F022FF
:0C151900ECF0A3EDF0A3EEF0A3EFF02245
:10152500A8828583F0D083D08212153C12153C1217
:10153500153C12153CE473E493A3C583C5F0C5833C
:10154500C8C582C8F0A3C583C5F0C583C8C582C810
:011555002273
:101FBF00AC6CAD6DAE6EAF6F780FEFA2E2EC20E6BA
:101FCF0001B35D5E5FF47004FCFDFEFFEF13FFEEE7
:101FDF0013FEED13FDEC13FCD8E08C6C8D6D8E6E43
:101FEF008F6FEE547FFE228E6C8F6DE4F56EF56F62
:011FFF0022BF
:10413900C3EE6480948040028007C3E49FFFE49E3D
:02414900FE2254
:10020C000232FAE493A3F8E493A34003F68001F2DC
:10021C0008DFF48029E493A3F85407240CC8C333F3
:10022C00C4540F4420C8834004F456800146F6DFC2
:10023C00E4800B0102040810204080903B73E47EA4
:10024C00019360BCA3FF543F30E509541FFEE493B7
:10025C00A360010ECF54C025E060A840B8E493A37E
:10026C00FAE493A3F8E493A3C8C582C8CAC583CAA9
:10027C00F0A3C8C582C8CAC583CADFE9DEE780BE61
:013BFB0000C9
:00000001FF
